:020000040000FA
:0200000047298E
:080008009100030E92008B1A17
:100010002D280B1A1D28120E8300910E110E0900B7
:1000200081018316640088308100831285140130B9
:10003000860090308B00900108008B100C308C00F3
:100040008C0B202806180B28AD30810020308B0047
:100050000230900008308C000B280B11101940283A
:100060008C0803193928060C8D0C8C03AD308100E7
:100070000B28061C5A28013090000D088E005A28C3
:1000800090195A288C08031952288F0C031C4B28EE
:10009000000085144E288510000000008C03B53048
:1000A00081000B2800000000000085149015A83086
:1000B00081000B2810308B00013090050B28851033
:1000C000063090000000B5308100A0308B00083071
:1000D0008C0008007420101C6A28101008005F2093
:1000E0007420901870280800080064309300000005
:1000F000000000000000000000000000930B7728C3
:100100000800061987281A1887281A149A158619BC
:100110008D289A188D289A149A11080014089600B0
:100120007520960B9028812008008E208E208E202E
:100130000800150896007520960B9B28080099204A
:10014000992099200800003097001B3084006A2015
:100150000E080D3C0319C7281708353C0319A728BA
:100160000E088000970A840AA728051585118E209D
:10017000051185158E201A101A160800051585110F
:100180009520051185158E209A101A1208001B3033
:10019000840097080319D8281018D828061DD828D5
:1001A000861DD828E020840A97030319D828CC2874
:1001B000003097001B30840072308F006F2056296A
:1001C00020308002031C08005B3000020318080086
:1001D00003308A00000880239800981B0229980D9C
:1001E0000830990003109903980D031CF328990B0C
:1001F000FA281029980D031CFE280029B520F7289D
:10020000BE20F72880301802031D0A299F209F2056
:1002100099200800FF301802031D0F29080008006C
:100220009F2008006A200E0894006A200E0895009E
:1002300072308F006F2056298312890183160814AB
:1002400083120808031956298F006F20890A1E2976
:100250008120061D861930291A151A1E41294329A5
:100260001A1D36291A1186182D2945291A189A1C83
:100270003C299A19432941291A1841299A184329D6
:100280004529B5202929BE2029299A01080083166D
:10029000FF30860000308500831285010511851529
:1002A000102040309400403095009A012821101C05
:1002B000562910100E083C3C0319A3280E083E3C9A
:0E02C000031912290E085E3C03191C29562949
:1007000082078034FF34FF34FF34FF34FF34FF347A
:10071000FF34FF34FF3445342A34733428345534DD
:1007200032343F342F3427342334213420343034CE
:1007300038343C343E343634FF34FF343134FF3403
:100740004C34FF34053418341A340C340234123467
:100750000E341034043417340D3414340734063492
:100760000F3416341D340A34083403340934113478
:100770000B3419341B341C34FF34FF34FF34FF3482
:10078000FF34FF34053418341A340C340234123474
:100790000E341034043417340D3414340734063452
:1007A0000F3416341D340A34083403340934113438
:0807B0000B3419341B341C3416
:02400E00F93F78
:10420000530065007200690061006C0020004300EB
:1042100057002000760031002E00310039002000C8
:1042200028006300290020003200300030003200F6
:1042300020006200790020004E004B003000450055
:044240000D0000006D
:00000001FF
